S01F00002E2E5C62696E5C64656D6F70726F675F786D63343730302E73726563E9
S3150800400000000220DD4A00082B4B00082D4B000853
S315080040102F4B0008314B0008334B00080000000006
S31508004020000000000000000000000000354B0008FA
S31508004030374B000800000000394B00086D4C00089B
S315080040403F4B0008414B0008434B0008454B00080E
S31508004050474B0008494B00084B4B00084D4B0008DE
S315080040604F4B0008000000000000000000000000A0
S31508004070514B000800000000534B0008554B000840
S31508004080574B0008594B00085B4B00085D4B00086E
S315080040905F4B0008614B0008634B0008654B00083E
S315080040A0674B0008694B00086B4B00086D4B00080E
S315080040B06F4B0008714B0008734B0008754B0008DE
S315080040C0774B0008794B00087B4B00087D4B0008AE
S315080040D07F4B0008814B0008834B0008854B00087E
S315080040E0874B0008894B00088B4B00088D4B00084E
S315080040F08F4B0008914B0008934B0008954B00081E
S31508004100974B0008994B00089B4B00089D4B0008ED
S315080041109F4B0008A14B0008A34B0008A54B0008BD
S31508004120A74B0008A94B0008AB4B0008AD4B00088D
S31508004130AF4B0008B14B0008B34B0008B54B00085D
S31508004140B74B0008B94B0008BB4B0008BD4B00082D
S31508004150BF4B0008C14B0008C34B0008C54B0008FD
S315080041600000000000000000000000000000000041
S31508004170C74B0008C94B0008CB4B0008CD4B0008BD
S31508004180CF4B0008D14B0008D34B0008D54B00088D
S31508004190D74B0008D94B0008DB4B0008DD4B00085D
S315080041A0DF4B0008E14B0008E34B0008E54B00082D
S315080041B0E74B0008E94B0008EB4B0008ED4B0008FD
S315080041C0EF4B0008F14B0008F34B0008F54B0008CD
S315080041D0F74B0008F94B0008FB4B000800000000ED
S315080041E0FD4B0008FF4B0008014C0008034C000873
S315080041F0054C000800000000074C000800000000FD
S31508004200EE11AA5510B5054C237833B9044B13B1F2
S315080042100448AFF300800123237010BD7C00002002
S3150800422000000000444D0008084B10B51BB10849B2
S315080042300848AFF300800848036803B910BD074B68
S31508004240002BFBD0BDE81040184700BF0000000057
S3150800425080000020444D000868000020000000008F
S31508004260154B002B08BF134B9D46A3F5803A00213A
S315080042708B460F461348144A121A00F039FD0F4BA5
S31508004280002B00D098470E4B002B00D098470020F3
S31508004290002104000D000D48002802D00C48AFF399
S315080042A0008000F0FFFC2000290000F00DFC00F063
S315080042B0E5FC00BF00000800000002200000000026
S315080042C0000000007C000020EC0000200000000038
S315080042D0000000002DE9F0438BB04FF461430193D1
S315080042E008238DF808308DF8093001258DF80A5015
S315080042F010278DF80B700026ADF80C601C4C01A930
S31508004300204600F0B9FA8DF81C6008954FF00209AE
S315080043108DF82490DFF85C8007AA0421404600F057
S3150800432025FA90238DF8103005958DF818900DEB29
S3150800433007020521404600F019FAE36923F007034E
S315080043402B43E3612B4604223946204600F01AFB2C
S315080043502B4604223146204600F02CFB236C23F022
S315080043600F0343EA090323640BB0BDE8F08300BFDB
S315080043700000034000810248074BD3F8143113F0BC
S31508004380080F07D110B50446034800F0A9FA2070B3
S31508004390012010BD002070470000034008B5FFF754
S315080043A099FF08BDBFF34F8F0549CA6802F4E0625A
S315080043B0044B1343CB60BFF34F8F00BFFDE700BF2D
S315080043C000ED00E00400FA0508B5174B1B785BB949
S315080043D01648FFF7D1FF012824D10122124B1A7083
S315080043E00022134B1A7008BD114B1B7801330F4876
S315080043F01844FFF7C1FF012814D10D4A1378013379
S31508004400DBB21370094A127893420BD10022064B8D
S315080044101A70064B5B78FF2B04D1044B9B780BB9BB
S31508004420FFF7C0FF08BD00BF990000209C000020D0
S315080044309800002008B5FFF7C7FF08BD10B5054C62
S3150800444080220821204600F0FFF94FF08073636050
S3150800445010BD00BF0085024808B500F001FC0D4BF1
S315080044601B68C31AB3F5FA7F13D30B4B1B783BB9FA
S315080044700122094B1A704FF48072084B5A6006E005
S315080044800022054B1A704FF08072044B5A60014B9C
S31508004490186008BDE0000020E400002000850248FE
S315080044A082B00023019303E000BF019B013301930F
S315080044B0019B8342F8D302B0704700BF72B60D4B1A
S315080044C00D4A9A60BFF34F8F62B6D3F8882042F43C
S315080044D07002C3F888205A6922F008025A6107490F
S315080044E041F214028B5823F00F0343F004038B5058
S315080044F0704700BF00ED00E00040000800100058BB
S3150800450000487047001BB70010B51E4BDB6813F454
S31508004510803F27D01C4BDB6813F0010F02D1FFF751
S31508004520EFFF00E01948184B1B6813F0040F11D071
S3150800453015498A68C2F303628B68C3F306238C683D
S31508004540C4F30644611C02FB0112B0FBF2F203FB42
S31508004550022208E00C4B9B6803F07F030133B0FB93
S31508004560F3F200E0094A0749C868C0B20130B2FB55
S31508004570F0F3086900F001000130B3FBF0F0044BDA
S31508004580186010BD004600501047005000366E01F6
S315080045906800002070B55F4B9A6842F04D029A6039
S315080045A04D22DA60A0331B6813F0010F09D15A4A6D
S315080045B0536843F001035360574B1B6813F0010F10
S315080045C0FAD0564B1B6813F4007F08D0534A9368F9
S315080045D043F40073936041F64C50FFF761FF504C6B
S315080045E0636843F40023636040F6C410FFF758FF7E
S315080045F0636823F4803323F002036360494B5B68E6
S3150800460013F0300F24D0103C636823F03003636046
S31508004610FFF776FF444BA3FB00231B0D013B6268A3
S3150800462042EA034363603E4BDA6822F00102DA602D
S315080046305A6822F400325A60394B1B6803F46073D7
S31508004640B3F5607FF8D1334A936823F0010393608A
S31508004650334B5A6842F001025A605A6842F0100217
S315080046605A60324A9A605A6842F040025A605A685A
S3150800467022F010025A605A6842F480225A60284B87
S315080046801B6813F0040FFAD0254A536823F0010378
S315080046905360234B1B6813F0010FFAD11D4A936828
S315080046A023F004039360224C4FF00113E3600026C5
S315080046B066612661266266620323E3611D4BA36178
S315080046C01D4BA362164D6B6823F040036B601B4BB2
S315080046D0AB604FF41660FFF7E3FE194BAB604FF47F
S315080046E06160FFF7DDFE174BAB604FF49650FFF79E
S315080046F0D7FE154BAB6041F27070FFF7D1FE134B36
S31508004700AB604FF4E150FFF7CBFE6660FFF7FCFEA7
S3150800471070BD00BF60410050004200500044005088
S3150800472010470050004700506BCA5F6B002F0B0103
S31508004730004600500500010003002001002F050176
S31508004740002F0301002F0201002F0101002F000195
S3150800475010B54FF00053044C0FCB84E80F00FFF759
S31508004760ADFEFFF717FF10BD6C000020F0B48B08F4
S315080047701F1D50F8276001F00305ED00F824AC4032
S3150800478026EA040440F82740466F4F000324BC403D
S3150800479026EA04044467194CA04203D004F5807441
S315080047A0A04207D1046E012606FA01F124EA0101A6
S315080047B0016617E054688C404460CC08103450F801
S315080047C0247001F00701890007268E4027EA0606AD
S315080047D040F8246050F82470167A06FA01F1394335
S315080047E040F82410043350F82340117801FA05F2F2
S315080047F0224340F82320F0BC704700BF008E0248D1
S31508004800020F20F07040034B53F822201368184318
S31508004810106070472C4D0008034B1868034B5B6902
S3150800482003F00103D8407047680000200046005096
S31508004830020F20F07040034B53F8222013681843E8
S31508004840106070471C4D000830B48B08043350F8CC
S31508004850235001F00301C900F8248C4025EA04041A
S3150800486040F8234050F823408A4044EA020140F8C1
S31508004870231030BC704700BF70B505460E4600F0E1
S31508004880E1F8F47904B9102422463168284600F084
S3150800489033F8B379013B64080134240244EA43033C
S315080048A043F00103EB633379013B1B0643F4817341
S315080048B06B6373792BB16A6B013B42EA03436B6303
S315080048C005E06A6B3379013B42EA03436B634FF4B5
S315080048D0A063AB634FF0FF33EB6433892B6470BD81
S315080048E0D0F80C3113F0E06F02D1406D80B27047FA
S315080048F0D0F81C0180B2704763293BD9002A3BD007
S315080049002DE9F04115460C460646FFF785FF1B497B
S31508004910A1FB00377F09A1FB0431480940F2FF3E9D
S315080049204FF0010CE046714611E007FB01F300FB6E
S3150800493005F2B3FBF2F39C0AC3F30903B4F5806FDF
S3150800494004D29E4502D99E46A446884601390029C6
S31508004950EBD148F4004333617269094B1340013DBA
S3150800496043EA85230CF1FF3C43EA0C4373610020BC
S31508004970BDE8F08101207047012070471F85EB5183
S31508004980EF8000FC30B4D0F8084124F0E064C0F8A9
S315080049900841D0F80851064C2C4041EA032343EA63
S315080049A0026244EA0203C0F8083130BC704700BF0F
S315080049B0C0C0FFF830B4D0F80C4124F0E064C0F869
S315080049C00C41D0F80C51074C2C4041EA032343EA2A
S315080049D0026244EA020343F08053C0F80C3130BC4B
S315080049E0704700BFC0C0FFEF10B5114B984208D101
S315080049F04FF40060FFF71CFF4FF40060FFF700FF5D
S31508004A0010BD0C4B984207D10B4C2046FFF710FF00
S31508004A102046FFF7F5FE10BD084B984206D1084C14
S31508004A202046FFF705FF2046FFF7EAFE10BD00BF48
S31508004A3008000340080002488000001008400248A9
S31508004A400001001010B50446154B984203D003F533
S31508004A500073984203D11348FFF7C6FF14E0124BC0
S31508004A60984203D003F50073984203D10F48FFF725
S31508004A70BBFF09E00E4B984203D003F5007398423A
S31508004A8002D10C48FFF7B0FF0323E360E36813F095
S31508004A90010FFBD0236C23F00F03236410BD00BF66
S31508004AA000000340080003400000024808000248CE
S31508004AB0004002480840024808B5FFF725FDFFF701
S31508004AC0BDFC00F0ABF808BD08B5FFF7F5FFFFF72A
S31508004AD065FCFFF7C1FCFFF7ADFCFAE707498D4611
S31508004AE00749084A084B9A42BEBF51F8040B42F8D8
S31508004AF0040BF8E7054880470548004700000220F0
S31508004B00504D0008000000206800002051470008AA
S31508004B10614200083C493D4A002301E041F8043B54
S31508004B209142FBD3FFF7D0FFFEE7FEE7FEE7FEE77D
S31508004B30FEE7FEE7FEE7FEE7FEE7FEE7FEE7FEE73F
S31508004B40FEE7FEE7FEE7FEE7FEE7FEE7FEE7FEE72F
S31508004B50FEE7FEE7FEE7FEE7FEE7FEE7FEE7FEE71F
S31508004B60FEE7FEE7FEE7FEE7FEE7FEE7FEE7FEE70F
S31508004B70FEE7FEE7FEE7FEE7FEE7FEE7FEE7FEE7FF
S31508004B80FEE7FEE7FEE7FEE7FEE7FEE7FEE7FEE7EF
S31508004B90FEE7FEE7FEE7FEE7FEE7FEE7FEE7FEE7DF
S31508004BA0FEE7FEE7FEE7FEE7FEE7FEE7FEE7FEE7CF
S31508004BB0FEE7FEE7FEE7FEE7FEE7FEE7FEE7FEE7BF
S31508004BC0FEE7FEE7FEE7FEE7FEE7FEE7FEE7FEE7AF
S31508004BD0FEE7FEE7FEE7FEE7FEE7FEE7FEE7FEE79F
S31508004BE0FEE7FEE7FEE7FEE7FEE7FEE7FEE7FEE78F
S31508004BF0FEE7FEE7FEE7FEE7FEE7FEE7FEE7FEE77F
S31508004C00FEE7FEE7FEE7FEE77C000020EC0000205A
S31508004C10014B1860704700BFE800002008B50C4B30
S31508004C201B680C4AA2FB03239B09013BB3F1807F57
S31508004C3009D2094A5360FC21084B83F82310002344
S31508004C409360072313600020FFF7E2FF08BD00BF4B
S31508004C5068000020D34D621010E000E000ED00E08F
S31508004C60014B1868704700BFE8000020024A136825
S31508004C7001331360704700BFE800002008B5074BF2
S31508004C80044613B10021AFF30080054B1868836A08
S31508004C9003B19847204600F033F800BF0000000033
S31508004CA0404D000870B50E4B0E4CE41AA4100025B2
S31508004CB01E46A54204D056F8253098470135F8E730
S31508004CC000F020F8084C094BE41AA41000251E46EB
S31508004CD0A54204D056F8253098470135F8E770BD47
S31508004CE060000020600000206400002060000020B2
S31508004CF002440346934202D003F8011BFAE77047C1
S31508004D00FEE70000F8B500BFF8BC08BC9E46704731
S31508004D10F8B500BFF8BC08BC9E4670474846005028
S31508004D2054460050604600506C46005014440050EB
S31508004D30204400502C4400503844005043000000E2
S30D08004D4000000020000000003D
S30D08004D4818F5FF7F01000000C9
S31508004D500000000000000000000000000000000045
S31508004D600000000000000000000000000000000035
S31508004D703C4D000800000000000000000000000094
S31508004D800000000000000000000000000000000015
S31508004D900000000000000000000000000000000005
S31508004DA000000000000000000000000000000000F5
S30D08004DB029420008054200082B
S31508004DB800000000000000000000000000000000DD
S30908004DC800000000D9
S70508004000B2
